:100000000C94E10E0C940B0F0C940B0F0C940B0F33
:100010000C940B0F0C940B0F0C940B0F0C940B0FF8
:100020000C940B0F0C940B0F0C944D910C94CA91E3
:100030000C940B0F0C940B0F0C940B0F0C940B0FD8
:100040000C940B0F0C94B0680C940B0F0C940B0FCA
:100050000C940B0F0C940B0F0C94967D0C94AC909D
:100060000C940B0F0C940B0F0C940B0F0C940B0FA8
:100070000C940B0F0C940B0F0C940B0F0C940B0F98
:100080000C940B0F0C940B0F0C940B0F0C940B0F88
:100090000C948B8B0C940B0F3B8E678E898E898E04
:1000A000898E898E898E898E898E898E898E898E98
:1000B000898E898E7F8E778E6F8E898E898E898EBE
:1000C000898E898E898E898E618E478E4F8E598E4C
:1000D0004E414E494E495459494E46CDCCCC3D0A2D
:1000E000D7233C17B7D13877CC2B329595E6241F10
:1000F000B14F0A000020410000C84200401C4620C9
:10010000BCBE4CCA1B0E5AAEC59D742020506C61FB
:100110006E6E657242756666657242797465733A91
:1001200020002046726565204D656D6F72793A201A
:1001300000436F6D70696C65643A204E6F762031B4
:100140003520323031380A00207C20417574686FC8
:10015000723A2044722E5068696C33440A0032307F
:1001600031382D30382D303100204C6173742055DA
:100170007064617465643A2000312E312E390A00B2
:100180004D61726C696E0020536F667477617265A1
:100190002052657365740A00205761746368646F48
:1001A000672052657365740A002042726F776E2073
:1001B0006F75742052657365740A00204578746504
:1001C000726E616C2052657365740A00506F7765BA
:1001D0007255700A0073746172740A005072696E0D
:1001E0007465722068616C7465642E206B696C6C38
:1001F00028292063616C6C6564210A004B494C4CD2
:1002000045442E20004B494C4C2063617573656456
:1002100020627920746F6F206D75636820696E614C
:1002200063746976652074696D65202D206375722D
:1002300072656E7420636F6D6D616E643A2000208C
:10024000746F6F206C6F6E67206578747275736958
:100250006F6E2070726576656E7465640A00206347
:100260006F6C6420657874727573696F6E2070723C
:100270006576656E7465640A006F6B005265736520
:100280006E643A2000416476616E6365204B3D00E8
:100290003F4B2076616C7565206F7574206F66200A
:1002A00072616E67652028302D3130292E0A003AA0
:1002B000200050726F6265205A204F666673657425
:1002C000003F5A206F7574206F662072616E6765FB
:1002D00020282D3520746F203230290A00454550E2
:1002E000524F4D204F4B0A00426564204C657665A5
:1002F0006C696E6720004661696C656420746F20CC
:10030000656E61626C6520426564204C6576656C43
:10031000696E670A00426564204C6576656C20430F
:100320006F7272656374696F6E204D617472697863
:100330003A004E6F2063617365206C696768740AC8
:100340000043290A0061626C656420286D696E2093
:1003500074656D702000436F6C64206578747275ED
:10036000646573206172652000496E76616C696412
:100370002065787472756465720A0020643A002002
:10038000693A0020703A0050726F6265205A204F1F
:1003900066667365743A200020466C6F773A2000D9
:1003A000205A00205900580020204D61783A200042
:1003B000205A00205900580020204D696E3A200034
:1003C0004F6666004F6E2000536F667420656E6442
:1003D00073746F70733A2000546F6F2066617220DF
:1003E00066726F6D207265666572656E63652070FA
:1003F0006F696E740A0020540020520041636365E7
:100400006C65726174696F6E3A2050002F2F200066
:100410003A004361703A00544845524D414C5F5098
:10042000524F54454354494F4E004155544F524545
:10043000504F52545F53445F5354415455530045F9
:100440004D455247454E43595F5041525345520026
:10045000434153455F4C494748545F4252494748DE
:10046000544E45535300544F47474C455F4C494702
:1004700048545300534F4654574152455F504F57CD
:100480004552004255494C445F50455243454E54F5
:10049000004C4556454C494E475F44415441005A33
:1004A0005F50524F4245004155544F4C4556454CC4
:1004B000005052494E545F4A4F420050524F4752EB
:1004C000455353004155544F5245504F52545F5479
:1004D000454D5000564F4C554D45545249430045EB
:1004E0004550524F4D0053455249414C5F584F4E75
:1004F0005F584F4646004649524D574152455F4E60
:10050000414D453A4D61726C696E20312E312E3964
:1005100020284769746875622920534F5552434516
:100520005F434F44455F55524C3A68747470733A58
:100530002F2F6769746875622E636F6D2F4D61721E
:100540006C696E4669726D776172652F4D61726C70
:10055000696E2050524F544F434F4C5F5645525393
:10056000494F4E3A312E30204D414348494E455F68
:10057000545950453A506C617920426F74204D6F48
:100580006465726E2045585452554445525F434F3E
:10059000554E543A3120555549443A343063653606
:1005A0003164312D326564302D343533302D38339C
:1005B00030342D3535653365656161656266660A7F
:1005C0000020573A006F6B004D3131332053004B00
:1005D000494C4C45442E20004543484F00494E4667
:1005E0004F004552524F52530044525952554E00FB
:1005F000434F4D4D554E49434154494F4E006F6650
:100600006600D805DD05E205E905F00544454255DB
:10061000473A0050726F7465637465642050696E68
:100620000A0000011C1D132FFFFFFFFF1E1F12FFFA
:1006300018FFFFFF20211124FFFFFFFFFFFFFF0E28
:1006400010FFFFFF22230DFFFFFF0E260F2C272593
:1006500069730025696D2025697300256968202567
:10066000696D202569730025696420256968202546
:10067000696D202569730025697920256964202525
:1006800069682025696D20256973005072696E7450
:100690002074696D653A2000205A3A200020593AAA
:1006A000200042656420583A20000A0A426564200E
:1006B0004C6576656C20436F7272656374696F6E0A
:1006C000204D61747269783A00202844525952557D
:1006D0004E2900473239204175746F2042656420ED
:1006E0004C6576656C696E67003F285629657262B5
:1006F0006F7365206C6576656C20697320696D7019
:100700006C61757369626C652028302D34292E0A5E
:1007100000496E76616C69642065787472756465F1
:10072000720A004163746976652045787472756455
:1007300065723A200020453A00205A3A0020593A82
:1007400000583A002C20002C2000486F6D6520587E
:10075000592066697273740A005761726E696E6718
:100760003A20486F6D696E672042756D702044694C
:100770007669736F72203C20310A000202046275B0
:1007800073793A2070617573656420666F722069B1
:100790006E7075740A00627573793A2070617573B2
:1007A000656420666F7220757365720A00627573E6
:1007B000793A2070726F63657373696E670A0050CF
:1007C000726F62696E67206661696C65640A0020F9
:1007D0005A3A200020593A200042656420583A20B5
:1007E000002066697273740A005A00590058004864
:1007F0006F6D65200020496E76616C6964206578B4
:1008000074727564657220004B494C4C45442E202F
:10081000005072696E7465722073746F70706564D5
:100820002064756520746F206572726F72732E205C
:1008300046697820746865206572726F7220616EF7
:100840006420757365204D39393920746F207265C5
:1008500073746172742E202854656D7065726174B2
:100860007572652069732072657365742E205365F7
:100870007420697420616674657220726573746196
:100880007274696E67290A004E6F20436865636B56
:1008900073756D2077697468206C696E65206E755C
:1008A0006D6265722C204C617374204C696E653AE0
:1008B0002000636865636B73756D206D69736D618E
:1008C0007463682C204C617374204C696E653A2007
:1008D000004C696E65204E756D62657220697320EB
:1008E0006E6F74204C617374204C696E65204E7578
:1008F0006D6265722B312C204C617374204C696ED3
:10090000653A20004D31313000656E717565756551
:10091000696E67202200FF01FF0000A0400000A0D8
:1009200040000000400000C84200003E43000003B9
:10093000430000000000003E43000000000000C82B
:100940004200003E4300000343000000000000009E
:100950000000000000000048420000484200008003
:1009600040000000003A0A0020286D6D2900202078
:100970004D393030204B004C696E65617220416406
:1009800076616E63653A0A0020204D383531205A71
:10099000005A2D50726F6265204F66667365740051
:1009A00020440020490020204D3330312050005099
:1009B00049442073657474696E67733A0A00202095
:1009C0004D3432302053004175746F2042656420ED
:1009D0004C6576656C696E673A0A00205A002059AA
:1009E0000020204D323036205800486F6D65206F52
:1009F00066667365743A0A00204500205A00205943
:100A00000020580020540020530020204D32303563
:100A100020510020453C6D61785F655F6A65726BAF
:100A20003E0020583C6D61785F785F6A65726B3E6E
:100A300020593C6D61785F795F6A65726B3E205A20
:100A40003C6D61785F7A5F6A65726B3E00416476E7
:100A5000616E6365643A20513C6D696E5F736567D2
:100A60006D656E745F74696D655F75733E20533C90
:100A70006D696E5F66656564726174653E20543CA5
:100A80006D696E5F74726176656C5F6665656472D0
:100A90006174653E0020540020520020204D323009
:100AA00034205000416363656C65726174696F6ED8
:100AB0002028756E6974732F7332293A20503C7068
:100AC00072696E745F616363656C3E20523C72654F
:100AD00074726163745F616363656C3E20543C743F
:100AE000726176656C5F616363656C3E0A002045E8
:100AF00000205A0020590020204D3230312058006B
:100B00004D6178696D756D20416363656C657261D7
:100B100074696F6E2028756E6974732F7332293A69
:100B20000A00204500205A0020590020204D323074
:100B3000332058004D6178696D756D206665656478
:100B400072617465732028756E6974732F73293A06
:100B50000A00204500205A0020590020204D39323B
:100B600020580053746570732070657220756E692B
:100B7000743A0A0020204D3230302044300A0020E0
:100B8000204D3230302044002044697361626C652E
:100B9000640A0046696C616D656E742073657474D7
:100BA000696E67733A002020473231202020203BB5
:100BB0000048617264636F646564204465666175B2
:100BC0006C742053657474696E6773204C6F616434
:100BD00065640A00DC050000DC050000DC0500009F
:100BE000102700000000FA420000FA420000A04076
:100BF0000000C8410000A0420000A0420080FC4468
:100C00000000BD42290A002062797465733B2063AD
:100C1000726320002073746F72656420736574744E
:100C2000696E6773207265747269657665642028E1
:100C300000202863616C63756C6174656429210A06
:100C40000020213D2000454550524F4D2043524346
:100C5000206D69736D61746368202D202873746F33
:100C60007265642920002053697A653A2000496E34
:100C70006465783A2000204D61726C696E3D56358E
:100C800035290A0028454550524F4D3D00454550F5
:100C9000524F4D2076657273696F6E206D69736D6A
:100CA000617463682000290A002062797465733BCF
:100CB00020637263200053657474696E67732053F8
:100CC000746F726564202800454550524F4D206472
:100CD00061746173697A65206572726F722E0A00A1
:100CE0004572726F722077726974696E6720746FD3
:100CF00020454550524F4D210A006F70656E0054DB
:100D00005249474745524544003A20007A5F6D6991
:100D10006E00795F6D617800785F6D696E00526575
:100D2000706F7274696E6720656E6473746F702083
:100D30007374617475730A00205A3A0020593A009E
:100D400020583A00656E6473746F7073206869741C
:100D50003A2000486F6D696E67206661696C656452
:100D600000556E6B6E6F776E20636F6D6D616E6494
:100D70003A20220020746F6F206C6F6E67206578B8
:100D800074727573696F6E2070726576656E7465C6
:100D9000640A0020636F6C642065787472757369EF
:100DA0006F6E2070726576656E7465640A00FFFD73
:100DB000FCFAF8F6F4F2F0EEECEAE9E7E5E3E1E05C
:100DC000DEDCDAD9D7D5D4D2D0CFCDCBCAC8C7C50F
:100DD000C3C2C0BFBDBCBAB9B7B6B4B3B2B0AFAD91
:100DE000ACAAA9A8A6A5A4A2A1A09E9D9C9A9998E8
:100DF0009795949392908F8E8D8B8A89888786841D
:100E0000838281807F7E7D7B7A7978777675747333
:100E10007271706F6E6D6C6B6A696867666564632A
:100E20006261605F5E5D5C5B5A5958585756555415
:100E300053525150504F4E4D4C4B4A4A49484746E9
:100E400046454443424241403F3E3E3D3C3B3B3AA7
:100E500039383837363535343332323130302F2E59
:100E60002E2D2C2B2B2A29292827272625252423FC
:100E70002322212120201F1E1E1D1C1C1B1B1A1992
:100E8000191818171616151514131312121111101C
:100E90000F0F0E0E0D0D0C0C0B0A0A09090808079E
:100EA0000706060505040403030202010000000012
:100EB00000010000000100008000555555000000B1
:100EC000400033333300AAAA2A00499224000000CC
:100ED0002000C7711C0099991900D145170055557C
:100EE00015003BB11300244912001111110000003C
:100EF00010000F0F0F00E3380E0043790D00CCCC2B
:100F00000C00C3300C00E8A20B0064210B00AAAA5D
:100F10000A00703D0A009DD80900427B0900922416
:100F20000900DCD30800888808001042080000008F
:100F30000800F0C107008787070075500700711C83
:100F400007003EEB0600A1BC06006990060066663D
:100F50000600703E06006118060017F4050074D103
:100F600005005BB00500B2900500627205005555A2
:100F7000050078390500B81E0500050505004EEC92
:100F8000040087D40400A1BD040090A70400499286
:100F90000400C17D0400EE690400C7560400444407
:100FA00004005C3204000821040041100400000029
:100FB00004003FF00300F8E0030026D20300C3C39F
:100FC0000300CCB503003AA803000A9B0300388E47
:100FD0000300C08103009F750300D0690300505EC9
:100FE00003001D53030034480300913D03003333D5
:100FF000030016290300381F030097150300300C67
:101000000300030303000BFA020049F10200BAE8EF
:1010100002005CE002002DD802002DD0020059C869
:101020000200B0C0020031B90200DAB10200AAAA7F
:101030000200A0A30200BC9C0200FA9502005C8F93
:101040000200DF88020082820200457C02002776CF
:10105000020027700200436A02007C640200D05E36
:1010600002003F590200C85302006563686F3A00EE
:101070004572726F723A00205A3A0020593A0020A5
:10108000436F756E7420583A00232C0000B822007C
:1010900000561800003A0F0000B8080000B1040024
:1010A00000710200003E01000024F4D43050C38ED1
:1010B00020C2A24017828B7011127A910D816CD9D7
:1010C0000AA861E108C7586607615143061E4B5DD7
:1010D00005C145A7041A411104093D98037139312E
:1010E000034036DB0265339102D4305402802E1D5A
:1010F00002632CEE01752AC501B028A001102781DA
:10110000018F2564012B244B01E0223401AC211F07
:10111000018D200D01801FFC00841EED00971DDF56
:1011200000B81CD200E61BC600201BBC00641AB22B
:1011300000B219A8000A19A0006A189900D11791E5
:101140000040178B00B516840031167E00B3157968
:10115000003A157300C7146F0058146A00EE136646
:10116000008813630025135E00C7125B006C1257E2
:101170000015125400C111510070114F0021114B84
:1011800000D61049008D104700461044000210425E
:1011900000C00F4000800F3E00420F3C00060F3B96
:1011A00000CB0E3800930E37005C0E3500270E344E
:1011B00000F30D3200C10D3100900D3000600D2E96
:1011C00000320D2D00050D2C00D90C2B00AE0C2982
:1011D00000850C29005C0C2700350C27000E0C261E
:1011E00000E80B2400C40B2400A00B23007D0B237C
:1011F000005A0B2100390B2100180B2000F80A1FA0
:1012000000D90A1E00BB0A1E009D0A1D00800A1D8F
:1012100000630A1C00470A1B002C0A1B00110A1A53
:1012200000F7091A00DD091900C4091900AB0919F2
:1012300000920917007B091800630917004C091672
:101240000036091600200916000A091500F50815D0
:1012500000E0081400CC081400B8081400A4081416
:1012600000900813007D0812006B08130058081244
:10127000004608120034081100230811001208115A
:101280000001081100F0071000E0071000D007105F
:1012900000C0071000B0070F00A107100091070E53
:1012A0000083070F0074070F0065070E0057070E35
:1012B0000049070E003B070D002E070E0020070D0A
:1012C0000013070D0006070D00F9060C00ED060DD2
:1012D00000E0060C00D4060C00C8060C00BC060C8E
:1012E00000B0060C00A4060B0099060C008D060B3E
:1012F0000082060B0077060B006C060B0061060AE5
:101300000057060B004C060A0042060A0038060A7F
:10131000002E060A0024060A001A060A0010060912
:101320000007060A00FD050900F4050900EB0509A0
:1013300000E2050900D9050900D0050900C7050923
:1013400000BE050900B5050800AD050800A50509A2
:10135000009C050800940508008C05080084050819
:10136000007C050800740508006C05070065050889
:10137000005D050700560508004E050700470507F4
:10138000004005080038050700310507002A050759
:1013900000230507001C050600160507000F0507BA
:1013A000000805060002050700FB040600F5040717
:1013B00000EE040600E8040600E2040700DB040671
:1013C00000D5040600CF040600C9040600C30406C5
:1013D00000BD040600B7040600B1040500AC040615
:1013E00000A6040600A00405009B04060095040561
:1013F00000900406008A04050085040500800406A8
:10140000007A04050075040500700405006B0405EE
:101410000066040500610405005C0405005704052E
:1014200000520405004D040500480405004304056E
:10143000003E0404003A04050035040500300404AD
:10144000002C04050027040400230405001E0404E6
:10145000001A04040016040500110404000D04041D
:1014600000090405000404040000040400FC030453
:1014700000F8030400F4030400F0030400EC030488
:1014800000E8030400E4030400E0030400DC0304B8
:1014900000D8030400D4030400D0030400CC0304E8
:1014A00000C8030300C503030024F404D9201BC4AF
:1014B0000C5C0E9804C4095F0265077101F405F91C
:1014C00000FB04B30048048700C1036900580355BA
:1014D0000003034500BE023A008402310053022A91
:1014E000002902250004022000E4011C00C80119A3
:1014F00000AF01170098011400840113007101105E
:10150000006101100051010E0043010D0036010B76
:10151000002B010B0020010B00150109000C010933
:101520000003010800FB000800F3000800EB0007BF
:1015300000E4000600DE000600D8000600D2000627
:1015400000CC000500C7000500C2000500BD000476
:1015500000B9000400B5000400B1000400AD0004AF
:1015600000A9000400A5000300A20003009F0004DE
:10157000009B000300980003009500020093000305
:1015800000900003008D0002008B00030088000221
:10159000008600020084000300810002007F000238
:1015A000007D0002007B000200790002007700014C
:1015B0000076000200740002007200010071000257
:1015C000006F0002006D0001006C0002006A000163
:1015D000006900020067000100660001006500016B
:1015E000006400020062000100610001006000016F
:1015F000005F0002005D0001005C0001005B000173
:10160000005A000100590001005800010057000174
:101610000056000100550001005400010053000075
:101620000053000100520001005100010050000170
:10163000004F0001004E0000004E0001004D00016F
:10164000004C0001004B0000004B0001004A00016B
:101650000049000100480000004800010047000167
:101660000046000000460001004500000045000162
:10167000004400010043000000430001004200005C
:101680000042000100410000004100010040000153
:10169000003F0000003F0001003E0000003E00014E
:1016A000003D0000003D0001003C0000003C000047
:1016B000003C0001003B0000003B0001003A00003C
:1016C000003A000100390000003900010038000034
:1016D000003800000038000100370000003700012A
:1016E0000036000000360000003600010035000022
:1016F0000035000000350001003400000034000017
:10170000003400010033000000330000003300010A
:101710000032000000320000003200010031000001
:1017200000310000003100010030000000300000F6
:1017300000300001002F0000002F0000002F0000EB
:10174000002F0001002E0000002E0000002E0001DE
:10175000002D0000002D0000002D0000002D0001D4
:10176000002C0000002C0000002C0000002C0001C8
:10177000002B0000002B0000002B0000002B0001BC
:10178000002A0000002A0000002A0000002A0001B0
:1017900000290000002900000029000000290000A5
:1017A0000029000100280000002800000028000097
:1017B000002800000028000100270000002700008A
:1017C000002700000027000000270001002600007D
:1017D0000026000000260000002600000026000170
:1017E0000025000000250000002500000025000065
:1017F0000025000000250001002400000024000056
:101800000024000000240000002400010023000048
:10181000002300000023000000230000002300003C
:10182000002300000023000100220000002200002D
:10183000002200000022000000220000002200011F
:101840000021000000210000002100000021000014
:101850000021000000210000002100010020000004
:1018600000200000002000000020000000200000F8
:10187000002000000020000000200001001F0000E8
:10188000001F0000001F0000001F0000001F0000DC
:10189000001F0000001F0001001E0000001E0000CD
:1018A000001E0000001E000000290A002028002958
:1018B00020453A0020280029205A3A0020280029F3
:1018C00020593A0020280020583A0053746570705F
:1018D00065722063757272656E742076616C7565D1
:1018E0007320696E20252028416D7073293A0A0003
:1018F00020403A00202F00546865726D616C2052C0
:10190000756E6177617900453120544845524D41EB
:101910004C2052554E41574159004B494C4C45447F
:101920002E2000202D20496E76616C696420657838
:10193000747275646572206E756D62657220210A1D
:101940000048656174696E67206661696C65640052
:1019500045312048656174696E67206661696C6510
:1019600064004D494E54454D502074726967676557
:10197000726564004531204572723A204D494E54DB
:10198000454D50004D415854454D50207472696783
:101990006765726564004531204572723A204D4199
:1019A0005854454D50006265640A002C20737973C9
:1019B00074656D2073746F70706564212048656173
:1019C0007465725F49443A20002CFFFFFFFFFF005F
:1019D000010101010123646566696E652044454685
:1019E00041554C545F4B64200023646566696E6505
:1019F0002044454641554C545F4B692000236465A3
:101A000066696E652044454641554C545F4B7020D5
:101A100000504944204175746F74756E6520666985
:101A20006E69736865642120507574207468652040
:101A30006C617374204B702C204B6920616E6420A4
:101A40004B6420636F6E7374616E74732066726F83
:101A50006D2062656C6F7720696E746F20436F6EC6
:101A600066696775726174696F6E2E680A00504905
:101A700044204175746F74756E65206661696C658C
:101A800064212074696D656F75740A00546865720D
:101A90006D616C2052756E6177617900453120541B
:101AA0004845524D414C2052554E415741590048EE
:101AB000656174696E67206661696C6564004531B3
:101AC0002048656174696E67206661696C656400B1
:101AD000504944204175746F74756E652066616964
:101AE0006C6564212054656D7065726174757265F2
:101AF00020746F6F20686967680A00204B643A2081
:101B000000204B693A2000204B703A20000A204305
:101B10006C617373696320504944200A0020547536
:101B20003A2000204B753A2000206D61783A200061
:101B3000206D696E3A200020643A200020626961BD
:101B4000733A2000504944204175746F74756E6576
:101B50002073746172740A00504944204175746F97
:101B600074756E65206661696C65642120426164EC
:101B7000206578747275646572206E756D62657229
:101B80000A0070012C0190012701B0012201C0015F
:101B90001D01F00118011002130130020E01600254
:101BA000090190020401C002FF000003FA00400393
:101BB000F5008003F000D003EB002004E600700481
:101BC000E100E004DC004005D700C005D20040067B
:101BD000CD00D006C8008007C3003008BE00F00862
:101BE000B900C009B400B00AAF00B00BAA00D00C15
:101BF000A500000EA000500F9B00C01096005012D0
:101C0000910000148C00C0158700B0178200B01935
:101C10007D00D01B7800001E730040206E009022D3
:101C20006900F024640040275F0090295A00E02BEF
:101C30005500102E500020304B0010324600E0338B
:101C4000410090353C001037370070383200A03921
:101C50002D00B03A2800A03B2300603C1E00103D40
:101C60001900903D1400103E0F00703E0A00C03E67
:101C70000500003F0000403FFBFF803FF6FFC03FF4
:101C8000F1FF0129022904290829102920294029C6
:101C90008029012C022C0126022604260826102663
:101CA000202640268026402C802C0123022304235A
:101CB0000823102320234023802301200220042016
:101CC00008201020202040208020102C202C012FC4
:101CD000022F042F082F102F202F402F802F7EFE41
:101CE0007EFD7EFB7EF77EEF7EDF7EBF7E7F000186
:101CF00000009F1D12000200005C1D430003000055
:101D0000581D04010309043E1D1802030904261D81
:101D10001603030904181D0C0C03310032003300B4
:101D20003400350000001603550053004200200027
:101D3000530065007200690061006C000000180328
:101D40005400650065006E00730079006400750042
:101D500069006E006F0000000403090409024300DB
:101D6000020100C032090400000102020100052442
:101D700000100105240100010424020605240600C8
:101D8000010705820308004009040100020A00005F
:101D9000000705030240000007058402400000120E
:101DA00001000202000020C0168304720201020337
:101DB000010001C102018036018136004B67A98A0A
:101DC000109511241FBECFEFD0E2DEBFCDBF12E0D1
:101DD000A0E0B1E0ECEAFFE301E00BBF02C0079036
:101DE0000D92A032B107D9F72EE0A0E2B2E001C017
:101DF0001D92AC30B207E1F71EE0C1EEDEE004C098
:101E00002197FE010E948595CE3DD107C9F70E941A
:101E1000CD8D0C94D49F0C9400004F925F926F92E2
:101E20007F928F929F92AF92BF92CF92DF92EF926A
:101E3000FF92CF934B015C0169017A0120E030E011
:101E400040EA51E40E94A7952B013C012FE632E1C4
:101E500043E85AEB0E94C19787FD48C023E830E071
:101E600048EC52E4C301B2010E941F9618160CF40C
:101E70003DC02FE632E143E85AEBC701B6010E94AC
:101E8000C19787FD33C022E430E04EE353E4C7013D
:101E9000B6010E941F9618164CF124EF3DEF4FE952
:101EA00051E4C501B4010E94C19787FD1FC023E81A
:101EB00030E044EB52E4C501B4010E941F961816AD
:101EC000ACF027EE3BEF4FE151E4C701B6010E94B1
:101ED000C19787FD0BC0C1E022E430E044E353E446
:101EE000C701B6010E941F9618160CF4C0E08C2F93
:101EF000CF91FF90EF90DF90CF90BF90AF909F90E9
:101F00008F907F906F905F904F900895FB010190AC
:101F10000020E9F73197AF01461B570BDC01ED912B
:101F2000FC910280F381E02D0994CF93DF931F92FF
:101F3000CDB7DEB76983DC01ED91FC910280F381BE
:101F4000E02D41E050E0BE016F5F7F4F09950F909B
:101F5000DF91CF910895FF920F931F93CF93DF935B
:101F6000F82E092F162FE2E1F4E06491EF0121969B
:101F7000662329F080E09EE0D8DFFE01F6CFEF2D4A
:101F8000F02F6491EF012196662329F080E09EE016
:101F9000CCDFFE01F6CFE0E1F4E06491EF012196A1
:101FA000662329F080E09EE0C0DFFE01F6CF412FDE
:101FB00050E060E070E080E09EE00E94148D6AE0F6
:101FC00080E09EE0DF91CF911F910F91FF90ADCF08
:101FD0004F925F926F927F92AF92BF92CF92DF92B9
:101FE000EF92FF92CF93DF93EB01FC01608171814F
:101FF000828193812CE3C22ED12CE12CF12CA701FC
:1020000096010E944795B62EA72ECA01B901A701D5
:1020100096010E9447956B017C01CA01B90128E134
:1020200030E040E050E00E9447952B013C01C9019F
:102030006DE671E00E94339561157105D9F0AF929C
:10204000BF92DF92CF925F924F929F938F937F9335
:102050006F9387E796E09F938F93DF93CF930E94D0
:10206000F29C8DB79EB70E960FB6F8949EBF0FBE2A
:102070008DBF61C00097C9F0AF92BF92DF92CF923F
:102080005F924F929F938F9387E696E09F938F93F3
:10209000DF93CF930E94F29CEDB7FEB73C960FB64C
:1020A000F894FEBF0FBEEDBF46C041145104610459
:1020B0007104B9F0AF92BF92DF92CF925F924F92CC
:1020C0008BE596E09F938F93DF93CF930E94F29CD2
:1020D0008DB79EB70A960FB6F8949EBF0FBE8DBF00
:1020E0002AC0C114D104E104F104A9F0AF92BF9257
:1020F000DF92CF9283E596E09F938F93DF93CF9308
:102100000E94F29CEDB7FEB738960FB6F894FEBF6A
:102110000FBEEDBF10C0AF92BF928FE496E09F93C9
:102120008F93DF93CF930E94F29C0F900F900F90AC
:102130000F900F900F90DF91CF91FF90EF90DF9075
:10214000CF90BF90AF907F906F905F904F90089529
:1021500081548A3108F040C0A82FB0E04091BF04FC
:102160005091C0046091C1047091C20404C076957E
:102170006795579547958A95D2F740FF2DC0E09116
:10218000CA04F091CB04AB55BB4F8C918823E1F08E
:10219000E80FF11D808190ED980F9A3080F08E321B
:1021A00029F4818180538A3078F409C08D3211F08E
:1021B0008B3251F4818190ED980F9A3018F49E2F54
:1021C0008F2F04C08E3251F090E080E09093C604CF
:1021D0008093C70481E0089580E008958281805350
:1021E0008A3090F7ECCFB4DF882341F081E0209172
:1021F000C6043091C704232B09F480E008950F939F
:102200001F93CF938091C6049091C704009711F15A
:10221000FC018F01C1912C2F2F7DA9F0C53411F045
:10222000C536B9F7F801108260E070E08091C6040D
:102230009091C7040E94A598F801C083562F472F9C
:10224000382F292F0BC060E070E0CF911F910F91C4
:102250000C94A59850E040E030E020E0652F742F0A
:10226000832F922FCF911F910F9108958091C604D3
:102270009091C704009731F04AE050E060E070E0D0
:102280000C940B9A60E070E0CB0108958091C60435
:102290009091C704009731F04AE050E060E070E0B0
:1022A0000C94339B60E070E0CB010895DFDF97FD75
:1022B0000AC0DCDF6F3F71058105910509F02CF440
:1022C000D5DF862F089580E008958FEF08958091DF
:1022D000C6049091C704892B31F0E8DF91E08111A9
:1022E00003C090E001C091E0892F08950F931F93E0
:1022F000CF93DF93CDB7DEB72C970FB6F894DEBF40
:102300000FBECDBFE3E8F4E080859185A285B3855B
:1023100044815581668177810081118122813381D9
:1023200009871A872B873C874D835E836F83788765
:1023300089839A83AB83BC83AE014F5F5F4FBE013D
:102340006B5F7F4FCE0109960E9488562FE834E0DC
:10235000AE014F5F5F4FBE016B5F7F4FCE010996AD
:102360000E94FB642C960FB6F894DEBF0FBECDBF63
:10237000DF91CF911F910F9108952F923F924F922D
:102380005F926F927F929F92AF92BF92CF92DF92B5
:10239000EF92FF920F931F93CF93DF93CDB7DEB7EA
:1023A00064970FB6F894DEBF0FBECDBF2A013B0184
:1023B000902EA12E6901082F10E0F801EA5EF64F79
:1023C000E491BB24B3941E160CF4B12CFF24F394B7
:1023D00020E030E0A901C301B2010E94C1971816A4
:1023E0000CF0F12C000F111F000F111FC8018D57A9
:1023F0009B4F1C01FC01108211821282138276DF36
:10240000F1014082518262827382E090A70220E053
:1024100030E0A901692D7A2DC6010E941F96811115
:1024200008C0F801EB5AF64F85919591A591B491AA
:1024300003C0892D9A2DD601898B9A8BAB8BBC8BCF
:1024400080918B0490918C04A0918D04B0918E04A6
:1024500040918704509188046091890470918A04A6
:1024600000918304109184042091850430918604A6
:102470000D871E872F87388B49875A876B877C8704
:102480008D839E83AF83B88719821A821B821C8238
:10249000AE014B5F5F4FBE01675F7F4FCE010D9670
:1024A0000E948856CE0101966C018E010F5E1F4F6F
:1024B0002FE834E0AE014B5F5F4FBE01675F7F4F97
:1024C0000C960E9419640E940958BF100E94444B48
:1024D00064960FB6F894DEBF0FBECDBFDF91CF91EB
:1024E0001F910F91FF90EF90DF90CF90BF90AF9032
:1024F0009F907F906F905F904F903F902F900895A6
:102500006FE874E083E00C942166CF93DF9300D0F2
:10251000CDB7DEB72091F20D3091F30DCE010196CB
:102520002115310529F48C509E409A83898304C07B
:10253000821B930B9A83898389819A810F900F90D4
:10254000DF91CF910895FF920F931F93CF93DF9365
:10255000FC0120812B3319F1D0916804D430F8F4B8
:10256000F62EBC01C09166040C2F10E0F0E6CF9F60
:10257000C00111248A519D4F0E94D29CF801EA5754
:10258000FD4FF082CF5FC43018F4C093660402C0E0
:1025900010926604DF5FD093680481E001C080E0A0
:1025A000DF91CF911F910F91FF900895EF92FF92CD
:1025B0001F93CF93DF937C0160E0C5DF182F882342
:1025C000C9F0EAE6F0E16491EF012196662329F073
:1025D00080E09EE0AADCFE01F6CFB70189E099E039
:1025E0000E944F6762E280E09EE09FDC6AE080E04C
:1025F0009EE09BDC812FDF91CF911F91FF90EF90A8
:102600000895DF92EF92FF920F931F93CF93DF9382
:10261000CDB7DEB76E970FB6F894DEBF0FBECDBF55
:102620006091E4027091E5026115710541F14DE19F
:1026300050E0CE0101967C010E94889C1E8EF7011D
:102640008F010E191F09D190DD2019F09AE0D912DF
:10265000F7CFF701E00FF11F1082C701A7DF882332
:1026600071F0DD20A9F00F5F1F4F8091E40290917F
:10267000E502080F191F1093E5020093E40281E0C0
:102680002091E4023091E502232B29F480E003C07D
:1026900000E010E0F0CF6E960FB6F894DEBF0FBEEC
:1026A000CDBFDF91CF911F910F91FF90EF90DF9001
:1026B0000895EF92FF920F931F93CF93DF937C01C6
:1026C00084E591DDD82F882369F1F0DDC82F181635
:1026D0002CF5EAE6F0E164918F010F5F1F4F66234E
:1026E00029F080E09EE021DCF801F5CF6DE480E088
:1026F0009EE01BDCA70160E070E020E080E09EE04F
:102700000E94B88C6C2FCC0F770B85EF97E00E945E
:1027100077676AE080E09EE008DC08C080939A0258
:10272000D0E004C08091A70280939A028D2FDF91A0
:10273000CF911F910F91FF90EF9008950F931F93EA
:10274000CF93DF9394E0899FE00111248E010A5416
:102750001D4FFE01EE53FD4FDE01A253BD4F2D91E3
:102760003D914D915C9160817181828193810E9444
:10277000A895F8016083718382839383FE01E75BF0
:10278000F64F85919591A591B491FE01E655FD4FC7
:1027900080839183A283B383FE01E35CF64F85912E
:1027A0009591A591B491C55FDE4F88839983AA83E3
:1027B000BB83DF91CF911F910F910895CF92DF924C
:1027C000EF920F931F93CF93DF93CDB7DEB7609750
:1027D0000FB6F894DEBF0FBECDBFE090A702E3E8CE
:1027E000F4E080859185A285B38544815581668119
:1027F000778100811181228133810D871E872F8788
:10280000388B49875A876B877C878D839E83AF83FC
:10281000B88719821A821B821C82AE014B5F5F4F00
:10282000BE01675F7F4FCE010D960E948856CE0194
:1028300001966C0109E111E02FE834E0AE014B5F35
:102840005F4FBE01675F7F4F0C960E9419646096D0
:102850000FB6F894DEBF0FBECDBFDF91CF911F91B1
:102860000F91EF90DF90CF9008954F925F926F920B
:102870007F928F929F92AF92BF92CF92DF92EF9210
:10288000FF920F931F93CF93DF93CDB7DEB72C97B3
:102890000FB6F894DEBF0FBECDBF6D837E838F83EE
:1028A000988729873A874B875C874701580136010B
:1028B0008091190190911A01A0911B01B0911C0106
:1028C00089839A83AB83BC83D601CD90DD90ED9054
:1028D000FC9020E030E0A901C701B6010E941F96DC
:1028E000811106C0EDE5F9E0C590D590E590F49032
:1028F000A501940160918B0470918C0480918D04EA
:1029000090918E040E941F9687FF11C0C0921901FA
:10291000D0921A01E0921B01F0921C0180928B046C
:1029200090928C04A0928D04B0928E0447DFF30144
:10293000408051806280738020E030E0A901C301B3
:10294000B2010E941F96811108C040900101509071
:1029500002016090030170900401409219015092AD
:102960001A0160921B0170921C018D819E81AF81C2
:10297000B8858093830490938404A0938504B093D6
:10298000860489859A85AB85BC858093870490935E
:102990008804A0938904B0938A0410DFA5019401F0
:1029A00060918B0470918C0480918D0490918E04C1
:1029B0000E94C19718168CF4C0921901D0921A0186
:1029C000E0921B01F0921C0180928B0490928C0487
:1029D000A0928D04B0928E04F1DE0E940958898184
:1029E0009A81AB81BC818093190190931A01A093C5
:1029F0001B01B0931C012C960FB6F894DEBF0FBEDE
:102A0000CDBFDF91CF911F910F91FF90EF90DF909D
:102A1000CF90BF90AF909F908F907F906F905F907E
:102A20004F900895CF92DF92EF92FF920F931F93F2
:102A30006B01FC01E080F18002811381E3E8F4E0A6
:102A400024813581468157816081718182819381A2
:102A50000CDF1F910F91FF90EF90DF90CF900895C2
:102A6000CF92DF92EF92FF920F931F936A01E09053
:102A70008B04F0908C0400918D0410918E04FB0166
:102A80002081318142815381FC0160817181828189
:102A90009381EBDE1F910F91FF90EF90DF90CF902D
:102AA00008958091190190911A01A0911B01B09194
:102AB0001C018093E0029093E102A093E202B093A4
:102AC000E30280911701909118019093DF028093A7
:102AD000DE0284E690E09093180180931701089538
:102AE0008091E0029091E102A091E202B091E302B4
:102AF0008093190190931A01A0931B01B0931C01BC
:102B00008091DE029091DF0290931801809317016B
:102B10000895EF92FF920F931F93CF93DF93882333
:102B200029F0D0917204D095D17001C0D0E0662315
:102B300041F01091720411FB882780F911E01827E9
:102B400001C010E0442341F0C0917204C2FB882709
:102B500080F9C1E0C82701C0C0E0D11105C0111142
:102B600003C0CC2309F457C0EAE6F0E164917F0189
:102B70008FEFE81AF80A662329F080E09EE0D5D9A5
:102B8000F701F4CFEFEEF7E064917F018FEFE81AE1
:102B9000F80A662329F080E09EE0C7D9F701F4CF58
:102BA000DD2371F0EDEEF7E064917F018FEFE81A1D
:102BB000F80A662329F080E09EE0B7D9F701F4CF48
:102BC000112369F0EBEEF7E064918F010F5F1F4F67
:102BD000662329F080E09EE0A8D9F801F5CFC11165
:102BE00003C0E1EEF7E00CC0E9EEF7E06491EF011D
:102BF00021966623B1F380E09EE097D9FE01F6CFDF
:102C00006491EF012196662329F080E09EE08DD942
:102C1000FE01F6CFC1E08C2FDF91CF911F910F9174
:102C2000FF90EF900895BF92CF92DF92EF92FF92C4
:102C30000F931F93CF93DF93CDB7DEB728970FB6CF
:102C4000F894DEBF0FBECDBF90919F04981709F492
:102C50007AC0B82E882309F453C080E090E0A0EA3F
:102C6000B0E48D839E83AF83B887C0909602D090E6
:102C70009702E0909802F090990220E030E0A901DC
:102C8000C701B6010E941F9687FF0CC0A7019601DD
:102C900060E070E080EA90E40E94A7956D837E83F7
:102CA0008F83988720E030E043E053E46D817E819C
:102CB0008F8198850E94C197181644F480E090E0B7
:102CC000A3E0B3E48D839E83AF83B88720918B0408
:102CD00030918C0440918D0450918E046D817E81E1
:102CE0008F8198850E94C197181654F419821A8210
:102CF0001B821C82BE016F5F7F4FCE01059692DE64
:102D0000609183047091840480918504909186047D
:102D100020918704309188044091890450918A045D
:102D200019821A821B821C82E0908B04F0908C0422
:102D300000918D0410918E04FE0131966F0195DD96
:102D40008B2D0E944F4B80E028960FB6F894DEBF83
:102D50000FBECDBFDF91CF911F910F91FF90EF90EC
:102D6000DF90CF90BF9008954F925F926F927F92C5
:102D70008F929F92AF92BF92CF92DF92EF92FF928B
:102D80000F931F93CF93C82FE82EF12CF701EA5E23
:102D9000F64FB490823021F481E045DF811107C104
:102DA0006701CC0CDD1CCC0CDD1CF601EB5DF64F95
:102DB00045905590659074906B2DBB0C770B880BEC
:102DC000990B0E94BE964B015C0120E030E040EC84
:102DD0005FE3C301B2010E94F597A50194010E942F
:102DE000F597AB01BC0100E010E098018C2FC5DA2B
:102DF000C23041F0F601E75EF64F259135914591DD
:102E0000549104C020E030E040E450E4C501B40136
:102E10000E94F5974B015C0120E030E0A9010E947F
:102E20001F96882309F45CC0C23021F000E010E056
:102E3000980104C000E010E020E830E4B501A401EE
:102E400070588C2F9ADAC23009F439C0F701E5586E
:102E5000F84F849181111DC0EAE6F0E164917F0191
:102E60008FEFE81AF80A662329F080E09EE05DD82B
:102E7000F701F4CFE9E5F7E064917F018FEFE81AFD
:102E8000F80A662329F080E09EE04FD8F701F4CFDE
:102E90008AE0F601EB5AF64F459055906590749094
:102EA000682F70E080E090E00E94BE969B01AC012C
:102EB000C301B2010E9423962B013C0105C0412CA5
:102EC000512C612C90E4792EA5019401C501B40127
:102ED0000E94A895AB01BC01930182018C2F4DDAB1
:102EE00081E090E00C2E01C0880F0A94EAF79091DF
:102EF0007104982B9093710490917204892B8093A4
:102F00007204F601E253FD4F108211821282138285
:102F10008C2F14DCF601EF5CF64F85919591A5910D
:102F2000B491F601ED57FB4F80839183A283B38365
:102F3000C230D1F4209196023091970240919802CC
:102F40005091990260918B0470918C0480918D0452
:102F500090918E040E94A79560938B0470938C04CB
:102F600080938D0490938E04C1D9F601ED58FB4FE8
:102F7000D601AD57BB4F8D919D910D90BC91A02D69
:102F800080839183A283B383C23089F480E0CF91A0
:102F90001F910F91FF90EF90DF90CF90BF90AF9077
:102FA0009F908F907F906F905F904F903CCECF918D
:102FB0001F910F91FF90EF90DF90CF90BF90AF9057
:102FC0009F908F907F906F905F904F900895AF92F9
:102FD000BF92CF92DF92EF92FF920F931F93CF9306
:102FE000DF938FEEA82E81E0B82E93E7E92E94E0D0
:102FF000F92E03E814E026EBC22E22E0D22EC0E028
:10300000D0E0F50181915F01A3D8882319F1F7D8A9
:10301000FE01E652FD4F2081211104C02091A6023D
:10302000222341F0F80120813181428153810E94A5
:10303000A8950AC0C330D10539F0F601208131814D
:10304000428153810E94A795F70160837183828337
:1030500093830AC0F80180819181A281B381F70135
:1030600080839183A283B3832196F4E0EF0EF11C59
:103070000C5F1F4F84E0C80ED11CC430D10509F08D
:10308000C0CF86E4B0D88823B9F0B9D820E030E0CA
:10309000A9010E94C19718167CF4B1D820E030E055
:1030A00040E752E40E9423966093190170931A013D
:1030B00080931B0190931C01DF91CF911F910F9181
:1030C000FF90EF90DF90CF90BF90AF900895CF9298
:1030D000DF92EF92FF920F931F93CF93DF930FB680
:1030E000F894C090F50DD090F60DE090F70DF090AB
:1030F000F80D0FBE8091A502811174C0809100016E
:10310000882309F46FC080918502882309F46AC07E
:1031100040918102509182026091830270918402F9
:1031200097018601041B150B260B370B37FD6DC06D
:10313000833031F134F481300CF454C0EAE6F0E12C
:1031400006C0843009F04EC0EAE6F0E133C0649175
:10315000EF012196662331F080E09EE00E94950FFA
:10316000FE01F5CFEDEAF7E06491EF0121966623C9
:1031700009F438C080E09EE00E94950FFE01F4CF74
:10318000EAE6F0E16491EF012196662331F080E0F8
:103190009EE00E94950FFE01F5CFE6E9F7E064910D
:1031A000EF0121966623F1F080E09EE00E94950FEA
:1031B000FE01F5CF6491EF012196662331F080E0A6
:1031C0009EE00E94950FFE01F5CFEEE7F7E06491D7
:1031D000EF012196662331F080E09EE00E94950F7A
:1031E000FE01F5CF2091000130E0A8EEB3E00E948F
:1031F0008E95C60ED71EE81EF91EC0928102D0928F
:103200008202E0928302F0928402DF91CF911F91BB
:103210000F91FF90EF90DF90CF9008950F931F9341
:10322000CF93DF9300D000D0CDB7DEB7809171048B
:1032300083708330E9F0EAE6F0E164918F010F5F7B
:103240001F4F662331F080E09EE00E94950FF80149
:10325000F4CFEAE4F7E064918F010F5F1F4F66231C
:1032600009F43DC080E09EE00E94950FF801F3CF85
:103270003DD880E090E0AEEBB2E480937704909389
:103280007804A0937904B0937A0480918B04909190
:103290008C04A0918D04B0918E0480937B04909354
:1032A0007C04A0937D04B0937E0480E090E0A0EFC6
:1032B000B1E48093730490937404A0937504B09365
:1032C000760419821A821B821C82AE014F5F5F4F07
:1032D00067E774E083E794E0C3DB82E045DD0F90AD
:1032E0000F900F900F90DF91CF911F910F91089544
:1032F0000F931F93CF93DF93CDB7DEB769970FB6C8
:10330000F894DEBF0FBECDBF0E9414776E8B7F8B0B
:10331000888F998FBE016F5F7F4FCE0146960E94C6
:10332000E80FEAE6F0E164918F010F5F1F4F66231B
:1033300031F080E09EE00E94950FF801F4CFBE01CD
:103340006F5F7F4F8BE896E00E944F676AE080E0F6
:103350009EE00E94950F69960FB6F894DEBF0FBEEF
:10336000CDBFDF91CF911F910F910895CF93DF9340
:10337000E0E7F0E16491EF012196662331F080E00F
:103380009EE00E94950FFE01F5CFE3E1F6E0649127
:10339000EF012196662331F080E09EE00E94950FB8
:1033A000FE01F5CFDF91CF91089588E690E081D9B5
:1033B000811122C08091930483FD1EC083E50E9489
:1033C000F3108823B9F00E94FF100E948B9670932F
:1033D0002E0D60932D0D80E00E948A7A0E94FF10CE
:1033E00020E030E04AEA52E40E941F96181614F0DA
:1033F0000E94BD760C941B670895CF93DF9389E6F6
:1034000090E057D9811116C0E5ECF5E06491EF0129
:103410002196662331F080E09EE00E94950FFE0128
:10342000F5CF0E94BB7E6AE080E09EE0DF91CF9105
:103430000C94950FDF91CF910895CF92DF92EF9288
:10344000FF9283E50E94F310882321F10E94561118
:103450008D3308F08CE38093DF0C0FB6F894C090A6
:10346000F50DD090F60DE090F70DF090F80D0FBE31
:10347000282F30E0A8EEB3E00E948E95C60ED71E2E
:10348000E81EF91EC092DB0CD092DC0CE092DD0C41
:10349000F092DE0CFF90EF90DF90CF90089580E5E2
:1034A0000E94F310811106C083E50E94F310882367
:1034B00059F005C00E94561181110CC0F5CF0E9431
:1034C00036116F3F710510F06FEF70E07093A90235
:1034D0006093A8020895DF92EF92FF920F931F93DB
:1034E000CF93DF9383E50E94A810882359F083E5EA
:1034F0000E94F310882319F00E94561101C080E049
:1035000080939304EAE6F0E16491EF01219666234B
:1035100031F080E09EE00E94950FFE01F5CFECE0D7
:10352000F6E06491EF012196662331F080E09EE0A1
:103530000E94950FFE01F5CF809193048823A9F195
:1035400082E0E82E86E0F82E00E010E020E0809196
:10355000930490E0002E02C0959587950A94E2F7B7
:1035600080FF1AC0DD24D394D20E222329F06CE20E
:1035700080E09EE00E94950FF70185919491FC01F7
:103580006491EC012196662331F080E09EE00E9478
:10359000950FCE01F4CF2D2D0F5F1F4FF2E0EF0EF0
:1035A000F11C0530110599F60DC0EEEFF5E06491C0
:1035B000EF012196662331F080E09EE00E94950F96
:1035C000FE01F5CF6AE080E09EE0DF91CF911F9190
:1035D0000F91FF90EF90DF900C94950FCF93DF93B6
:1035E00083E50E94F310882351F00E9456118D3319
:1035F00008F08CE380930001DF91CF910895EAE613
:10360000F0E16491EF012196662331F080E09EE0C5
:103610000E94950FFE01F5CF4091000150E060E05F
:1036200070E088EC95E00E94D5676AE080E09EE05B
:10363000DF91CF910C94950F4F925F926F927F9292
:10364000AF92BF92CF92DF92EF92FF920F931F93B0
:10365000CF938FEEA82E81E0B82E04E715E0C0E0EE
:10366000F50181915F010E94A810882309F46DC0C3
:10367000C33009F063C00E94FF106B017C0120E0A1
:1036800030E040EA51E40E941F9687FF4EC0A70138
:1036900096016091800570918105809182059091DD
:1036A00083050E9423962B013C019B01AC01609194
:1036B0004C0570914D0580914E0590914F050E94EB
:1036C000F59760934C0570934D0580934E0590934C
:1036D0004F05A30192016091900570919105809131
:1036E0009205909193050E94F597609390057093D1
:1036F000910580939205909393056091A405709134
:10370000A5058091A6059091A7050E94BC96A301EE
:1037100092010E94F5970E9490966093A405709381
:10372000A5058093A6059093A705C0928005D09229
:103730008105E0928205F092830507C00E94FF1088
:10374000F8016083718382839383CF5F0C5F1F4F87
:10375000C43009F085CFCF911F910F91FF90EF906A
:10376000DF90CF90BF90AF907F906F905F904F9021
:103770000C94F7660F931F93CF93DF93C3E8D4E0C5
:1037800006EB12E0F801208131814281538168818A
:1037900079818A819B810E94A895AB01BC0181E45B
:1037A00097E00E94B467F8012481358146815781F2
:1037B0006C817D818E819F810E94A895AB01BC01A7
:1037C0008DE397E00E94B467F8012085318542853A
:1037D0005385688579858A859B850E94A895AB016C
:1037E000BC0189E397E00E94B4674C855D856E85D6
:1037F0007F8585E397E00E94B467DF91CF911F91A9
:103800000F910C94D5744F925F926F927F928F922A
:103810009F92AF92BF92CF92DF92EF92FF920F935F
:103820001F93CF93DF938FEEC82E81E0D82E9EECAE
:10383000E92E92E0F92E00E010E0C0E0D0E0F601C1
:1038400081916F010E94F310882309F44DC00E94FA
:10385000FF104B015C01C33059F0F801EA54FD4FF1
:1038600020813181428153810E94A7954B015C01E7
:10387000F801ED57FB4F2081318142815381C50111
:10388000B4010E94A7952B013C012DEB37E346E8DC
:1038900055EB0E94C19787FD0AC02DEB37E346E840
:1038A00055E3C301B2010E941F961816ECF4C33011
:1038B00051F480928F0490929004A0929104B0925F
:1038C0009204D1E011C0A3019201F70160817181DE
:1038D000828193810E94A895F7016083718382831E
:1038E00093838C2F0E949E13CF5FF4E0EF0EF11CA8
:1038F0000C5F1F4FC43009F0A2CFD1110E9480127B
:10390000DF91CF911F910F91FF90EF90DF90CF90BB
:10391000BF90AF909F908F907F906F905F904F90EF
:1039200029CFCF93DF93E6EFF4E06491EF01219686
:10393000662331F080E09EE00E94950FFE01F5CFF6
:1039400060E086EE94E00E94AB0F61E08FED94E0C2
:103950000E94AB0F61E084ED94E00E94AB0F61E048
:1039600084EC94E00E94AB0F60E08BEB94E00E944B
:10397000AB0F61E081EB94E00E94AB0F61E087EA5E
:1039800094E00E94AB0F61E08FE994E00E94AB0FDE
:1039900061E081E994E00E94AB0F60E083E894E08D
:1039A0000E94AB0F60E084E794E00E94AB0F60E000
:1039B00086E694E00E94AB0F60E080E594E00E9410
:1039C000AB0F60E08FE394E00E94AB0F60E08AE20F
:1039D00094E00E94AB0F61E087E194E0DF91CF912A
:1039E0000C94AB0FFF920F931F93CF93DF93C09173
:1039F000C804D091C90483E0F12C40E08150D1F09B
:103A00009881292F2B7F2134C9F729812133B1F7E0
:103A1000913421F0953421F441E002C0FF24F39465
:103A20009E012E5F3F4FE9012F5F3F4F98819032FB
:103A3000D1F3E4CF442371F0EAE6F0E164918F0121
:103A40000F5F1F4F662331F080E09EE00E94950FCC
:103A5000F801F4CFFF2071F0ECE0F4E064918F0105
:103A60000F5F1F4F662331F080E09EE00E94950FAC
:103A7000F801F4CFBE0180E09EE00E94860F6AE06C
:103A800080E09EE0DF91CF911F910F91FF900C9409
:103A9000950FCF9388EC90E00E945913811140C09C
:103AA00084E40E94A8108823C1F10E94FF10C1E0A5
:103AB00020E030E0A9010E941F96811101C0C0E002
:103AC000C093CC04CC2349F10E94FF10E0919A02EC
:103AD00024E0E29FF0011124E45CFA4F60837183DB
:103AE0008283938320E030E0A90160913C057091CE
:103AF0003D0580913E0590913F050E941F968111E2
:103B00000CC080E090E0A0EEBFE380933C05909372
:103B10003D05A0933E05B0933F05CF910C942356ED
:103B2000CF910895CF9383E50E94F3108823A1F0ED
:103B30000E94FF1060935C0570935D0580935E05A5
:103B400090935F05609354057093550580935605D7
:103B500090935705C0E001C0C1E080E50E94F310DA
:103B6000882359F00E94FF1060935C0570935D05F7
:103B700080935E0590935F05C0E082E50E94F3109C
:103B8000882359F00E94FF106093580570935905DF
:103B900080935A0590935B05C0E084E50E94F31082
:103BA000882359F00E94FF106093540570935505C7
:103BB00080935605909357052CC0CC2351F140912A
:103BC0005C0550915D0560915E0570915F058CEF1D
:103BD00093E00E94B4674091580550915905609157
:103BE0005A0570915B0589EF93E00E94B46740919C
:103BF000540550915505609156057091570586EF13
:103C000093E00E94B4676AE080E09EE0CF910C945C
:103C1000950FCF91089581E50E94A810882351F057
:103C20000E944611609394057093950580939605C4
:103C30009093970583E50E94A810882351F00E9475
:103C4000FF10609360057093610580936205909307
:103C5000630584E50E94A810882351F00E94FF109C
:103C600060935005709351058093520590935305CE
:103C700088E50E94A810882351F00E94FF106093ED
:103C8000400570934105809342059093430589E573
:103C90000E94A810882351F00E94FF1060934405F1
:103CA0007093450580934605909347058AE50E94E9
:103CB000A810882351F00E94FF106093480570936C
:103CC000490580934A0590934B0585E40E94A8100E
:103CD000882351F00E94FF1060934C0570934D05AE
:103CE00080934E0590934F050895EF92FF920F93A6
:103CF0001F93CF938FEEE82E81E0F82E02EC12E0B6
:103D0000C0E0F70181917F010E94A810882351F043
:103D10000E94FF10F80160837183828393838C2F4C
:103D20000E949E13CF5F0C5F1F4FC33051F7CF919E
:103D30001F910F91FF90EF901DCDCF93DF93EAE697
:103D4000F0E16491EF012196662331F080E09EE07E
:103D50000E94950FFE01F5CF83E50E94A8108823ED
:103D600021F00E94671180930A01E8ECF3E064916E
:103D7000EF012196662331F080E09EE00E94950FCE
:103D8000FE01F5CF80910A01811103C0E0ECF3E060
:103D900002C0E4ECF3E06491EF012196662331F078
:103DA00080E09EE00E94950FFE01F5CFE8EBF3E086
:103DB0006491EF012196662331F080E09EE00E943D
:103DC000950FFE01F5CF2091B6023091B7024091D8
:103DD000B8025091B9026091AA027091AB02809131
:103DE000AC029091AD020E94A895AB01BC0186EB9C
:103DF00093E00E94B4672091BA023091BB024091D7
:103E0000BC025091BD026091AE027091AF028091F0
:103E1000B0029091B1020E94A895AB01BC0183EB66
:103E200093E00E94B4672091BE023091BF0240919E
:103E3000C0025091C1026091B2027091B3028091B0
:103E4000B4029091B5020E94A895AB01BC0180EB31
:103E500093E00E94B467E8EAF3E06491EF012196F1
:103E6000662331F080E09EE00E94950FFE01F5CFC1
:103E70002091B6023091B7024091B8025091B90238
